:020000040800F2
:10000000F8DA0120A10100087D2B0008C1240008B6
:10001000692B0008AD080008E53A00080000000060
:10002000000000000000000000000000A9340008EB
:100030009D1B000800000000E12C000801360008AC
:10004000BB010008BB010008BB010008BB010008A0
:10005000BB010008BB010008BB010008BB01000890
:100060003D1C00086D1C0008811C0008BB01000835
:10007000BB010008BB010008BB010008BB01000870
:10008000BB010008BB010008BB010008BB01000860
:10009000BB010008BB010008BB010008B11C00083F
:1000A000BB010008BB010008BB010008BB01000840
:1000B000BB0100086D360008BB010008BB01000849
:1000C000BB010008BB010008BB010008BB01000820
:1000D000BB010008BB010008BB010008BB01000810
:1000E000A11B0008BB010008BB010008BB01000800
:1000F000BB010008BB010008BB010008BB010008F0
:10010000BB010008BB010008BB010008BB010008DF
:10011000BB010008BB010008BB010008BB010008CF
:10012000BB010008BB010008BB010008BB010008BF
:10013000BB010008BB010008BB010008BB010008AF
:10014000BB010008BB010008BB010008BB0100089F
:10015000BB010008BB010008BB010008A137000873
:10016000BB010008BB010008BB010008BB0100087F
:10017000BB010008BB010008BB010008BB0100086F
:10018000BB010008BB010008DFF810D000F046F802
:1001900000480047B93C0008AFF30080F8DA0120BE
:1001A0000648804706480047FEE7FEE7FEE7FEE711
:1001B000FEE7FEE7FEE7FEE7FEE7FEE7053600089E
:1001C0008901000840EA01039B0703D009E008C940
:1001D000121F08C0042AFAD203E011F8013B00F80C
:1001E000013B521EF9D27047D2B201E000F8012B58
:1001F000491EFBD270470022F6E710B513460A46A7
:1002000004461946FFF7F0FF204610BD421C10F8C7
:10021000011B0029FBD1801A70470000064C074DD6
:1002200006E0E06840F0010394E8070098471034C6
:10023000AC42F6D3FFF7ACFFDC3E0008FC3E000802
:1002400070B58C1810F8015B15F0070301D110F898
:10025000013B2A1106D110F8012B03E010F8016BC5
:1002600001F8016B5B1EF9D12B0705D40023521E48
:100270000DD401F8013BFAE710F8013BCB1A921CB0
:1002800003E013F8015B01F8015B521EF9D5A142AE
:10029000D8D3002070BD70B506460C46154608E060
:1002A0003046721C96B200F007F804F8010B681E85
:1002B00085B2002DF4D170BD2DE9F0410446002532
:1002C000002702F025FBA02002F0EEFA02F072FBFC
:1002D000054605B129E0201202F0E6FA02F06AFBB9
:1002E000054605B121E02646E11704EB116109122C
:1002F000A4EB0121C8B202F0D7FA02F05BFB05467D
:1003000005B112E002F004FBA12002F0CDFA02F0E8
:1003100051FB054605B108E0002002F08FFA0746C0
:1003200002F01CFB3846BDE8F08102F017FB00200C
:10033000F9E72DE9F04105460C46164600270CE08A
:100340002178284600F010F80746012F02D000203F
:10035000BDE8F081681C85B2641C301EA6F1010165
:100360008EB2EDD10120F3E72DE9F04104460E46AF
:10037000002702F0CDFAA02002F096FA02F01AFB54
:100380000746201202F090FA02F014FB07462546B9
:10039000E11704EB11610912A4EB0121C8B202F0CC
:1003A00083FA02F007FB0746304602F07DFA02F0BE
:1003B00001FB074602F0D2FA0F2003F0C3FB012035
:1003C000BDE8F0811CB502F0E3F901211F2002F025
:1003D00025FF0620009001208DF8040000208DF8F4
:1003E000060003208DF8050001208DF807006946FE
:1003F0002A4801F0C4FE4FF4604000906946284846
:1004000001F0BDFE4FF4E05000906946254801F030
:10041000B6FE43F6010000906946234801F0AFFEA6
:1004200041F2100000906946204801F0A8FE042126
:100430001A4801F01AFF4FF40051194801F015FF56
:100440000121194801F011FF4FF48051164801F0C5
:100450000CFF4FF48051154801F007FF02210F48AF
:1004600001F003FF1021114801F0FFFE02201049A6
:100470000860012100F01CFA0421002000F018FAA5
:1004800047F6FF7001F014FD47F6FF7001F026FDFE
:1004900000F0C0F802F06EF81CBD00000000024041
:1004A0000004024000080240000C0240001002401C
:1004B0008C0000201CB50121102002F0AFFE0420AA
:1004C000009001208DF8040000208DF80600032024
:1004D0008DF8050001208DF807006946034801F0FA
:1004E0004EFE012002F036F81CBD00000010024054
:1004F00010B5002440480078012819D13F48006811
:1005000020F0FF003D4908603D48407809680843F5
:100510003A49086001213B48007800F0C9F90421FC
:100520003648006800F0C4F90020334908700124FF
:100530003548007801281AD13048006820F47F40FF
:100540002E4908602E484078096841EA00202B496E
:10055000086001212B48007800F0AAF904212748FF
:10056000006800F0A5F900202749087001242748F9
:10057000007801281AD12148006820F47F001F4923
:1005800008601F484078096841EA00401B4908603C
:1005900001211C48007800F08BF9042117480068FD
:1005A00000F086F9002019490870012418480078E5
:1005B00001281AD11148006820F07F400F490860D7
:1005C0000F484078096841EA00600C490860012141
:1005D0000C48007800F06CF904210848006800F02D
:1005E00067F900200A4908700124012C02D1642017
:1005F00003F0C8FA10BD0000900000209800002011
:10060000F3000020940000209100002092000020C0
:100610009300002000B585B00820009000208DF8E0
:10062000040003208DF8050002208DF807006946BC
:10063000334801F0A4FD4FF4006000906946314852
:1006400001F09DFD4FF48070009069462E4801F046
:1006500096FD2020009069462C4801F090FD012174
:10066000880302F0EBFD0B21022002F01FFF08219E
:10067000032002F01BFF0321002002F017FF0521D9
:10068000042002F013FF40F62810029000208DF89D
:100690000C0008208DF80D0001208DF80E0002A836
:1006A00001F0BCFB09208DF8100001208DF811002D
:1006B00000208DF8120001208DF8130004A802F02C
:1006C0005FFA17208DF8100001208DF811008DF8C9
:1006D00012008DF8130004A802F052FA28208DF8B9
:1006E000100001208DF8110003208DF81200012068
:1006F0008DF8130004A802F043FA05B000BD000015
:100700000000024000080240000C024000100240BD
:100710002DE9FF5F05460C462F78EE782879697938
:1007200000EB01201FFA80F8A879E97900EB01209D
:100730001FFA80F98DF808608DF80B40ADF809803C
:1007400001208DF80C0001AADDE9020101F06CFE28
:1007500083469DF80410584600F074FE8DF808603A
:100760008DF80B40ADF8099000208DF80C00012C9D
:1007700000D100BF022C00D100BF6A46DDE90201B2
:1007800001F052FE82469DF80000032802DB9DF82E
:10079000000000909DF80010504600F053FE2246E5
:1007A0003946022001F024F9BDE8FF9F01461329D4
:1007B00001DA00207047A1F109000A2290FBF2F350
:1007C00002FB130008B10020F4E70120F2E700006B
:1007D0002DE9FE4F04460D46277894F8018094F8E1
:1007E000029094F803A0207A617A00EB01201FFAAE
:1007F00080FB002000908DF80880ADF804B08DF8E3
:1008000009908DF807708DF806A0012D00D100BF6A
:100810006A46DDE9010101F02BFD06460EB9BDE88F
:10082000FE8F681EC100009888400549096808438A
:1008300003490860042D00D100BF00BFEFE70000AE
:10084000880000202DE9F04105462F781548006802
:1008500000F00040134908600026002410E047FA29
:1008600004F000F0010050B1621CD1B206EB860327
:100870006A1C02EB4300FFF7ABFF701CC6B2641C9E
:10088000042CECDB01210848006800F011F8042179
:100890000448006800F00CF8022003F053F9BDE8AA
:1008A000F0810000880000208C00002000BFFEE7DF
:1008B0002DE9F04104460E4600250027012E2BD1DC
:1008C00000BF26E004F0800747B14FF48051324862
:1008D00001F0CBFC012003F055F907E04FF4805103
:1008E0002D4801F0C0FC012003F04CF94FF4804189
:1008F0002A4801F0BAFC012003F044F94FF480418A
:10090000264801F0B0FC012003F03CF96400681CAB
:10091000C5B2082DD6DB3CE0042E3AD1002526E0F6
:1009200004F0004747B14FF480511B4801F09DFC93
:10093000012003F027F907E04FF48051164801F039
:1009400092FC012003F01EF94FF48041134801F09E
:100950008CFC012003F016F94FF480410F4801F0A0
:1009600082FC012003F00EF96400681CC5B2202D42
:10097000D6DB4FF40041094801F077FC012003F079
:1009800001F94FF40041054801F06DFC012003F02E
:10099000F9F8BDE8F08100000008024000040240C0
:1009A0002DE9F84380468946012505F108063046C1
:1009B00003F0CCF904467720009023462A46694686
:1009C000012000F089FC07463946204602F0BAFFB4
:1009D000204603F023F9BDE8F8832DE9F05F812775
:1009E000B946484603F0B2F9044639462046FFF7B7
:1009F00002FC07F1080A504603F0A8F9804601F00E
:100A00005BFD05462878207068786070A878A07033
:100A1000002004E0291D0A5CC11C6254401C0E2801
:100A2000F8DB05F11200FFF7F1FB0646102E01DDA1
:100A3000102000E030460646002006E005F11201D5
:100A40000A5C00F111016254401CB042F6DB05F172
:100A50002200FFF7DBFB0646202E01DD202000E010
:100A600030460646002006E005F122010A5C00F14E
:100A700021016254401CB042F6DB05F14200FFF751
:100A8000C5FB0646402E01DD402000E0304606460C
:100A9000002006E005F142010A5C00F141016254C8
:100AA000401CB042F6DB43463A462146022000F0A5
:100AB00013FC83465946404602F044FF404603F08B
:100AC000ADF8204603F0AAF8BDE8F09F2DE9F04FFD
:100AD000A9B08127B946484603F038F9044639469B
:100AE0002046FFF788FB07F1080A504603F02EF96D
:100AF0008046684603F0BAF86D462878207068781A
:100B00006070A878A070002004E0291D0A5CC11C58
:100B10006254401C0E28F8DB05F11200FFF776FB4B
:100B20000646102E01DD102000E03046064600206B
:100B300006E005F112010A5C00F111016254401C4B
:100B4000B042F6DB05F12200FFF760FB0646202EDF
:100B500001DD202000E030460646002006E005F1D9
:100B600022010A5C00F121016254401CB042F6DB14
:100B700005F14200FFF74AFB0646402E01DD40200A
:100B800000E030460646002006E005F142010A5C1E
:100B900000F141016254401CB042F6DB43463A4644
:100BA0002146022000F098FB83465946404602F059
:100BB000C9FE404603F032F8204603F02FF829B072
:100BC000BDE8F08F2DE9F04FA9B082468B460E2488
:100BD0002746384603F0BAF8054604F108084046AF
:100BE00003F0B4F80646684603F040F822460DF1DB
:100BF0008A012846FFF7E6FA3346224629460420B2
:100C000000F06AFB81464946304602F09BFE3046C2
:100C100003F004F8284603F001F829B0BDE8F08F8E
:100C200003F038F8012080F3138800BF00BFBFF342
:100C30004F8F0748006800F4E06006490843001D34
:100C400003490860BFF34F8F00BF00BFFEE70000FD
:100C50000CED00E00000FA0530B5A9B004460D46E1
:100C6000684603F003F80E2221460DF18A00FFF7D3
:100C7000A9FA684603F004F829B030BD70B50446FF
:100C80000D46902000F0BAFB70BD70472DE9F04F83
:100C900089B004460E464B48007810B109B0BDE853
:100CA000F08F012047490870324621464648FFF739
:100CB00089FA3046FFF77AFD30B9002041490870C3
:100CC000052000F09BFBE9E7A6F10800C5B2281D4E
:100CD00000F0FF09615D681C205C01EB0021A81C8D
:100CE000205C01EB0041E81C205C01EB00600790F8
:100CF00014F8091009F10100205C01EB002080B21A
:100D000006902946204601F001FC05902946204620
:100D100001F012FC824605990798884202D1069894
:100D2000504506D0002027490870FF2000F066FBE0
:100D3000B4E74FF0000B207804902046FFF782FDC7
:100D4000D84615E0049840FA08F000F0010068B1B8
:100D500008F10102D1B20BEB8B03621C02EB4300E2
:100D6000FFF7D6FC0BF1010000F0FF0B08F10108C2
:100D7000B8F1040FE6DB02200390039808300890D6
:100D8000089802F0E3FF0746002006E0B11E014488
:100D9000615C02AA1154411CC8B20228F6DB3B4632
:100DA00002A92220039A00F097FA0190384601998F
:100DB00002F0C8FD002003490870384602F02EFFFB
:100DC00000BF6BE784000020C4CE01202DE9F04174
:100DD00005460E46304601F0E7F820B9052000F040
:100DE0000DFBBDE8F0812F7800240DE047FA04F0F8
:100DF00000F0010038B1621CD1B204EBC4036A1CDC
:100E0000981801F081F8641C042CEFDB00BFE8E7C0
:100E10002DE9F041054688462E780027002420E081
:100E200046FA04F000F00100D0B1012000EB84008C
:100E3000285C00F00101022000EB8400285C61F3D3
:100E40005F10074632463946042000F0D1FD0420E9
:100E500000EB84002F5C32463946052000F0C8FDC7
:100E6000641C042CDCDB00F0DBFABDE8F081000040
:100E70002DE9F05F83460826B046404602F066FF43
:100E8000044606F10809484602F060FF0746154887
:100E9000008885B2280A207065701348008885B2E2
:100EA000280AA070E5701148008885B2280A2071D0
:100EB00065710F48008885B2280AA071E5713B462C
:100EC00032462146302000F007FA82465146384625
:100ED00002F038FD384602F0A1FE204602F09EFEE8
:100EE000BDE8F09FAC000020AE000020B000002064
:100EF000B200002070B504460D46902000F07EFA46
:100F000070BD2DE9F0479AB007460D46012D03D07C
:100F1000052000F073FA1DE0642606F1080840463B
:100F200002F014FF044601A9384601F0DAFE064635
:100F300001F0ABFE82462346324601A9332000F081
:100F4000CBF981464946204602F0FCFC204602F0DF
:100F500065FE00BF1AB0BDE8F08770B504460D46C7
:100F6000207802F01BF970BD2DE9F04105460E46D0
:100F7000052E04DA052000F041FABDE8F0812F7853
:100F800001200C49087000240DE047FA04F000F03D
:100F9000010038B1601CC1B2681C00F075F90A206C
:100FA00002F0F0FD641C042CEFDB00200149087006
:100FB00000BFE2E7840000202DE9F04105460E461F
:100FC000052E04DA052000F019FABDE8F0810120B1
:100FD00004E0295C01EB0727411CC8B20528F8DBB7
:100FE0002878801FC4B224B90121384600F018FBCC
:100FF00005E0012C03D10221384600F011FB022C40
:1010000003D10321384600F00BFB00BFDDE72DE9DB
:10101000F04105460E46022E04DA052000F0EEF9F6
:10102000BDE8F0816F782C78012C05D1012239467A
:10103000022000F0DDFC16E0022C05D10222394628
:10104000104600F0D5FC0EE0042C05D103223946F1
:10105000022000F0CDFC06E0082C04D10422394621
:10106000022000F0C5FC142002F08CFD00BFD7E781
:101070002DE9F04104460F46062F04DA052000F062
:10108000BDF9BDE8F0816078217800EB01250026EC
:10109000022004E0215C01EB0626411CC8B20628B0
:1010A000F8DB07490D700748066001212846FFF765
:1010B000FFFB04213046FFF7FBFB00BF00BFE0E76A
:1010C000940000209800002070B505460C46122CB4
:1010D00003DA052000F092F970BD1221284601F0D4
:1010E000CBFC00BFF8E7000070B59AB006460C468E
:1010F000072C04DA052000F081F91AB070BD1648FB
:10110000007800B1F9E7012013490870652C0ADA6C
:10111000002004E0FF2122180DF80210401CC4F149
:1011200065018142F6DC224631466846FFF74AF8FF
:101130000DF10101684601F029FE0546012D02D19D
:1011400000F06EF902E0FF2000F058F9002002499B
:10115000087000BFD1E700008400002038B50446C5
:101160000D4600F05DF902F027FE0020009038BD2A
:1011700000F056F900BFFEE72DE9F05F80468B4690
:10118000022698F8000020B1012804D0022806D1D8
:1011900003E0292604E0082602E0082600E000BF5C
:1011A00000BF3546284602F0D1FD044606F1080985
:1011B000484602F0CBFD07464946FF223846FFF776
:1011C00013F898F8000020B1012808D0022814D1A3
:1011D0000CE0312213492046FEF7F4FF0EE01248DE
:1011E0000068206011480068606007E010480068EF
:1011F000206010480068606000E000BF00BF3B4610
:1012000032462146E32000F067F8824651463846D0
:1012100002F098FB384602F001FD204602F0FEFC89
:10122000BDE8F09FC4CE0120240100202801002049
:1012300028020020240200202DE9F05F07468B469B
:101240008024A046404602F081FD054604F10809CD
:10125000484602F07BFD0646802239462846FEF7C6
:10126000B1FF334622462946E42000F035F8824695
:101270005146304602F066FB304602F0CFFC28466D
:1012800002F0CCFCBDE8F09F2DE9FE4304460D467C
:1012900026786778A078E17800EB01201FFA80F8C3
:1012A0000EB9012600E000268DF800708DF803507D
:1012B000ADF801808DF8046002AADDE9000101F0BB
:1012C000B3F881469DF80810484600F0BBF80120AD
:1012D00002F038FCBDE8FE832DE9F04106460F46DA
:1012E00015461C4655202070AA206070BB20A070B7
:1012F000E6702571280A6071002D04DD2A46394602
:10130000A01DFEF75FFF0D21A81D21540A21E81D35
:101310002154401CBDE8F0812DE9F04132483349A9
:10132000098830F811504FF6FF70854201D1BDE8B1
:10133000F0814FF6FF702C492C4A128821F81200D8
:1013400000200CE02A49495D2A4A1154691C44F2E4
:10135000080291FBF2F302FB13118DB2401CB0F5B1
:10136000026FEFDB23480078552807D121484078E9
:10137000AA2803D11F488078BB2800D0D7E71D4E8C
:10138000B088801D3146085C0D2804D1B088C01D8E
:10139000085C0A2800D0CAE713481449098830F8C5
:1013A000115012480088401C142190FBF1F201FBFF
:1013B00012000E4908800F4F002410E00E4810F86C
:1013C0003400F978884208D1B9880B4800EBC40092
:1013D00042680848801D904703E0601CC4B21E2C80
:1013E000ECDB00BF00BFA2E77CC60120200100208B
:1013F00074860120A4C601202C0100207FB505467B
:10140000FF208DF80C008DF80D006B46022203A919
:10141000FFF762FF04462146684602F093FA7FBD5B
:101420001FB5C0208DF80C008DF80D006B46022210
:1014300003A9FFF751FF04462146684602F082FAED
:101440001FBD00002DE9F04704460E460027B846B0
:101450000025A946012E04D0022E19D0032E48D112
:1014600030E001216B4800F0FEFE012002F08AFB13
:101470000121684800F0F9FE012002F083FB012100
:10148000644800F0F0FE012002F07CFB012531E011
:101490004FF40051604800F0E6FE012002F072FBBC
:1014A0004FF400515C4800F0E0FE012002F06AFBBE
:1014B0004FF40051584800F0D6FE012002F062FBC4
:1014C000022517E00421554800F0CDFE012002F06E
:1014D00059FB0421514800F0C8FE012002F052FBE4
:1014E00004214E4800F0BFFE012002F04BFB032513
:1014F00000E000BF00BF4FF4C051474800F0B5FE08
:10150000012002F03FFB4FF40061434800F0ABFEC6
:10151000012002F037FB4FF480513F4800F0A3FE5A
:10152000012002F02FFB00274AE04FF000082AE0DC
:1015300004F00049B9F1000F08D04FF400613648BB
:1015400000F093FE012002F01DFB07E04FF4006164
:10155000314800F088FE012002F014FB4FF4805166
:101560002D4800F082FE012002F00CFB4FF4805168
:10157000294800F078FE022002F004FB640008F124
:10158000010000F0FF08B8F1080FD1DB4FF4006153
:10159000214800F068FE012002F0F4FA4FF4805177
:1015A0001D4800F062FE012002F0ECFA4FF4805179
:1015B000194800F058FE022002F0E4FA781CC7B285
:1015C000042FB2DB4FF48051134800F04EFE01208F
:1015D00002F0D8FA4FF400610F4800F046FE0120F7
:1015E00002F0D0FA012D03D101210A4800F03DFE9E
:1015F000022D03D12903084800F037FE032D03D143
:101600000421064800F031FE012002F0BBFA00255B
:10161000BDE8F087000C02400004024000000240D8
:101620002DE9F04704460D460027C4F3034848F06F
:101630003009A6B2012D04D0022D04D0032D06D10D
:1016400003E0182705E01A2703E01C2701E0BDE8A6
:10165000F08700BF00F0F8FF384600F0C1FF01F04E
:101660003FF800B149E0484600F0BAFF01F038F811
:1016700000B142E0300A00F0B3FF01F031F800B1F0
:101680003BE0F0B200F0ACFF01F02AF800B134E02A
:1016900001F000F8012D04D0022D0ED0032D26D12B
:1016A00019E00121174800F0DEFD052002F06AFA7A
:1016B0000121144800F0D9FD1AE04FF400511248FE
:1016C00000F0D1FD052002F05DFA4FF400510E4804
:1016D00000F0CBFD0CE004210C4800F0C4FD052017
:1016E00002F050FA0421094800F0BFFD00E0AEE727
:1016F00000BF012002F026FAA9E700F0CBFF00BFEF
:10170000A5E70000000C0240000402400000024077
:1017100010B500241448006820F4401012490860F5
:1017200008460068086004E0601CC4B2012002F0B2
:1017300029FA0E48006808B1C82CF5DBC82C01DB7B
:10174000012010BD002404E0601CC4B2012002F09E
:1017500019FA0648006808B9F02CF5DBF02C01DB1B
:101760000120EEE70020ECE7000802402802414299
:1017700010B5002400F0B0F800F08CF8FFF7C8FFB7
:10178000CC2000F0B5F8BE2000F0B2F800F03CF834
:1017900004B2200104B22046E11704EB11710C11D0
:1017A00001480480204610BDAC0000201CB540F26A
:1017B0000140009001208DF8040000208DF8060003
:1017C00002208DF8050001208DF8070069460B48BE
:1017D00000F0D5FC4FF4007000906946084800F016
:1017E000CEFC4FF4007000906946064800F0C7FC3C
:1017F00000F050F8FFF78CFF1CBD0000000802400D
:10180000000C02400010024070B50026002408E0E1
:1018100000F00CF8054605FA04F0304386B2601C6F
:10182000C4B20C2CF4DB304670BD000010B50024AF
:101830001548006820F44010134908600846006805
:1018400040F480100860002010490860022002F077
:1018500099F901200E49C1F8A8020B48006820F44C
:101860004010094908600846006808600C2002F032
:1018700089F906488038006800B10124322002F05E
:1018800081F9204610BD000000080240A802414234
:101890000000414210B50D48006820F440100B498B
:1018A00008600846006840F480100860002008497D
:1018B000086040F2EE2002F065F901200549C1F808
:1018C000A8020F2002F05EF910BD000000080240DF
:1018D000A80241420000414210B5FFF7DBFFFFF7CD
:1018E00017FFCC2000F004F8442000F001F810BDF0
:1018F00070B504463648006820F44010344908604A
:101900000846006840F4801008603248006820F4FF
:101910004020304908600846006840F48020086094
:101920002D48006820F440202B49086008460068D4
:1019300040F4802008602648006820F00300244915
:1019400008600846006840F00100086001253CE09E
:1019500004F001066410DEB100202049086020492F
:10196000C1F8A4021F4908601F49C1F88002022083
:1019700002F008F90120194908601C49086019495A
:1019800008601949C1F880023C2002F0FBF81AE017
:101990000020124908601249C1F8A40211490860E8
:1019A0001149C1F880023C2002F0ECF801200B49FB
:1019B00008600E4908600B4908600B49C1F88002B5
:1019C000022002F0DFF8681CC5B2082DC0DD70BD32
:1019D00000080240000C024000100240A8024142F0
:1019E00000804142A402424200004142A48241429E
:1019F0002DE9F04707460E46904600250024B946DB
:101A0000B8F1010F09D0B8F1020F0DD0B8F1030FF2
:101A100011D0B8F1040F1AD113E04FF480515C4893
:101A200000F023FC012413E04FF48051594800F0EA
:101A30001CFC03240CE00221574800F016FC05248E
:101A400006E01021534800F010FC062400E000BF1F
:101A500000BF022002F096F8012C04D121034C486B
:101A600000F001FC14E0032C05D14FF480514948EB
:101A700000F0F9FB0CE0052C04D10221464800F0EF
:101A8000F2FB05E0062C03D11021424800F0EBFBED
:101A9000022002F077F800252BE009F0800ABAF165
:101AA000800F08D14FF40061394800F0DEFB0220BE
:101AB00002F068F807E04FF40061354800F0D3FB0E
:101AC000022002F05FF84FF40051314800F0CDFBE6
:101AD000022002F057F84FF400512D4800F0C3FBEC
:101AE000022002F04FF84FEA49604FEA1069681C83
:101AF000C5B2082DD1DB002529E006F0800ABAF135
:101B0000800F08D14FF40061214800F0AEFB0220A5
:101B100002F038F807E04FF400611D4800F0A3FB25
:101B2000022002F02FF84FF40051194800F09DFBFD
:101B3000022002F027F84FF40051154800F093FB03
:101B4000022002F01FF87006060E681CC5B2082DB0
:101B5000D3DB012C03D121030D4800F086FB032CBD
:101B600004D14FF480510B4800F07FFB052C03D1CA
:101B70000221094800F079FB062C03D11021054809
:101B800000F073FB022001F0FDFFBDE8F0870000CC
:101B9000000C0240001002400000024070470000AC
:101BA00010B54FF4806000F02DF9012814D11420F5
:101BB00001F0C8FF4FF400411B4800F04BFB30B967
:101BC0001A480078012802D10020184908704FF403
:101BD000806000F011F925E04FF4805000F012F918
:101BE000012814D1142001F0ADFF4FF480511048AA
:101BF00000F030FB30B90F480078012802D10020F6
:101C00000C4908704FF4805000F0F6F80AE04FF4E9
:101C1000006000F0F7F8012804D107490870C002FD
:101C200000F0EAF810BD0000000C0240A9000020FE
:101C300000000240A80000209000002010B51420F1
:101C400001F080FF0421074800F004FB30B906488A
:101C50000078012802D1002003490870042000F018
:101C6000CBF810BD000C0240A700002010B50120E9
:101C700002490870082000F0BFF810BD9200002053
:101C800010B5142001F05EFF1021074800F0E2FAC1
:101C900030B906480078012802D1002003490870B5
:101CA000102000F0A9F810BD000C0240A600002092
:101CB00010B5402000F0A6F8012812D1142001F040
:101CC00041FF4021124800F0C5FA30B911480078B0
:101CD000012802D100200F490870402000F08CF844
:101CE00015E0202000F08EF8012805D10A4908707F
:101CF000202000F081F80AE04FF4807000F082F8B4
:101D0000012804D105490870000200F075F810BDE3
:101D1000000C0240A500002093000020910000204C
:101D20000EB50121880301F089FA0221032001F098
:101D3000BDFB0421032001F0B9FB0621032001F0C3
:101D4000B5FB0821032001F0B1FB0A21002001F0BE
:101D5000ADFB0C21002001F0A9FB0521042001F0BE
:101D6000A5FB41F27450009000208DF8040008207B
:101D70008DF8050001208DF80600684600F04EF849
:101D800008208DF8080001208DF8090002208DF848
:101D90000A0001208DF80B0002A800F0F1FE0A20D5
:101DA0008DF8080002208DF8090001208DF80A0046
:101DB0008DF80B0002A800F0E3FE28208DF8080043
:101DC00003208DF8090002208DF80A0001208DF80B
:101DD0000B0002A800F0D4FE17208DF808000420A4
:101DE0008DF8090002208DF80A0001208DF80B0003
:101DF00002A800F0C5FE0EBD014908607047000052
:101E0000143C014001460020034A12680A400AB10E
:101E1000012000E000207047143C014000212349CC
:101E20008279002A3AD00A46126803689A430B4620
:101E30001A600A1D126803689A430B1D1A60027922
:101E400011440A6803681A430A60184A0832126883
:101E500003689A43154B08331A601A1D1268036809
:101E60009A43124B0C331A604279102A0ED11A1F72
:101E7000126803681A430D4B08331A601A1D126862
:101E800003681A43094B0C331A600DE00749427985
:101E900011440A6803681A430A6005E00279114494
:101EA0000A6803689A430A6070470000003C0140DA
:101EB0002DE9F041054602260C274FF00108064C9B
:101EC00044EA076444EA08442C4331462046FFF7BD
:101ED000B9FABDE8F0810000000030102DE9F041B2
:101EE000054602260C274FF00308064C44EA076417
:101EF00044EA08442C4331462046FFF7A3FABDE8E4
:101F0000F0810000000030102DE9FF5F0446657885
:101F1000A678E77894F808802079617900EB0120B1
:101F20001FFA80F9A079E17900EB01201FFA80FA0D
:101F300000201B4908601B480068019000200090A9
:101F40008DF80C508DF80D608DF80A708DF80E80AC
:101F50006B4601AADDE9020100F01EFA8346BBF1DF
:101F6000000F01D1BDE8FF9F9DF800000C490860FB
:101F70000C4901980860012109480068FEF798FCA7
:101F8000042108480068FEF793FC4846FFF7A6FFC7
:101F90005046FFF78DFF022001F0D4FD00BFE1E7BE
:101FA0008C0000208800002001460A2901DA002068
:101FB0007047481E092290FBF2F302FB130008B1A0
:101FC0000020F5E70120F3E70149086070470000B1
:101FD0000C3C024030B10749096841F48061054A70
:101FE000116005E00349096821F48061014A11602C
:101FF00070470000003C024070B504460A460026C7
:10200000092502B909E0012A01D1160205E0022AD8
:1020100001D1160201E04FF4407600F09FF805462A
:10202000092D28D11548006820F440701349086034
:1020300008460068304308600846006820F0F80051
:1020400008600846006844F0020108430B49086034
:102050000846006840F48030086000F07FF80546CC
:102060000648006820F0020004490860084600683D
:1020700020F0F8000860284670BD0000103C0240C7
:1020800009201349096801F48031B1F5803F01D17D
:1020900001201CE00E49096801F0100109B1062079
:1020A00015E00B49096801F4807109B102200EE0C6
:1020B0000749096801F0EF0109B1072007E0044969
:1020C000096801F0020109B1082000E00920704709
:1020D0000C3C02400348006840F0004001490860A1
:1020E00070470000103C024030B502460C460925FE
:1020F00000F034F80546092D19D10E48006820F487
:1021000040700C4908600846006840F400700860A0
:102110000846006840F001000860146000F01EF8F6
:1021200005460448006820F001000249086028467E
:1021300030BD0000103C02400548006800F000403F
:1021400028B1044802490C39086003480860704708
:10215000103C024023016745AB89EFCD08B509204B
:102160000090FFF78DFF009002E0FFF789FF0090DD
:102170009DF800000128F8D09DF8000008BDF0B5DA
:102180000A4600210023002400BF3DE0012505FA96
:1021900001F3156805EA03049C4234D105684F0039
:1021A0000326BE40B543056015794E00B54006686C
:1021B000354305601579012D02D01579022D16D110
:1021C00085684F000326BE40B543856055794E00B3
:1021D000B540866835438560456801268E40B54325
:1021E0004560456896798E40B6B235434560C5680E
:1021F0004F000326BE40B543C560D5794E00B540BB
:10220000C6683543C560491C1029BFD3F0BDF0B581
:10221000002300244D07ED0E02FA05F3CE1000F165
:10222000200555F826504E07F70E0F26BE40B54341
:10223000CF1000F1200646F82750CE1000F12005FF
:1022400055F8265045EA0304CE1000F1200545F864
:102250002640F0BD0246002013690B400BB101205F
:1022600000E0002070474183704701837047000001
:1022700017B500210023BDF800004FF6FF74A042FF
:1022800003D14348007801431BE0BDF80000B0F5DE
:102290007A7F03D13E484078014312E0BDF8000048
:1022A000B0F5FA7F03D13A488078014309E0BDF8E0
:1022B0000000142803D13648C078014301E0002013
:1022C0001EBD9DF8050038B99DF80200012803D114
:1022D00030480078014318E09DF8050038B99DF8B2
:1022E000020020B92B484078014301230DE09DF8FE
:1022F0000500012807D19DF8020020B92548807803
:102300000143012301E00020DAE7F3B19DF8040066
:10231000012802D09DF8040000B935E09DF80400C2
:10232000142802D141F008012EE09DF80400052890
:1023300002D141F0400127E09DF80400642802D159
:1023400041F0480120E00020BAE79DF80400012890
:1023500002D09DF8040000B916E09DF8040005289D
:1023600002D141F008010FE09DF80400142802D1C9
:1023700041F0480108E09DF80400642802D141F0D2
:10238000480101E000209BE71160012098E7000070
:10239000F3000020F00000200FB502219DF8060098
:1023A00000F0010008B141F080019DF8050000B97E
:1023B0001BE09DF80500012802D141F0080114E05E
:1023C0009DF80500022804D1106840F0004010601C
:1023D0000BE09DF80500032804D1106880F0004050
:1023E000106002E0002004B000BD9DF8020001284A
:1023F00002D141F0400105E09DF8020000B901E082
:102400000020F0E79DF80400012800D108E09DF8C5
:102410000400052802D141F0200101E00020E2E79C
:1024200019700120DFE70000F7B5042503269DF8A9
:102430000470012F01D1022501261D489DF800706E
:102440000FB92F4600E0374639469DF803707F1ECE
:10245000C7EB0717DFF85CC0674401EB410C17F8C6
:102460000C707F1F17709DF803707F1EC7EB071756
:10247000DFF840C0674401EB410C6744BB789DF82E
:1024800003707F1EC7EB0717DFF828C0674401EB16
:10249000410C67447C7840EA036040EA0440BDF8A0
:1024A000017038431778012F00D100BFFEBD000036
:1024B00000003010B40000200048704700000020E9
:1024C00002480349086000BFFEE700000400FA0567
:1024D0000CED00E0002111E00846082208E000F0C1
:1024E00001031BB1074B83EA500000E04008521E75
:1024F000002AF4DC044B43F82100491CFF29EBDDE2
:10250000704700002083B8ED3402002030B5024649
:102510000B464FF0FF31002008E0CCB2155C6C4058
:10252000044D55F8244084EA1121401C9842F4D30C
:10253000C84330BD3402002010B5024600230020FD
:1025400003E0145C1C44A3B2401C8842F9D3184633
:1025500010BD000010B50446012C04D1042104482C
:10256000FFF783FE03E004210148FFF77CFE10BD66
:10257000001002401CB50121022000F04FFE4FF474
:10258000C050009001208DF8040000208DF8060056
:1025900003208DF8050001208DF8070069460B48DF
:1025A000FFF7EDFD01200A4908600A49C1F8AC02B5
:1025B00001210948FFF759FE4FF400510348FFF786
:1025C00054FE04210548FFF750FE1CBD00040240E4
:1025D000B082404200804042000C024000000240B5
:1025E00070B504461548006820F44000134908609F
:1025F0000846006840F48000086000201049086028
:10260000002517E0E0090E49091F08606006040E66
:10261000022001F0B7FA01200A49C1F8B0020220F5
:1026200001F0B0FA002006490860022001F0AAFA81
:10263000681CC5B2082DE5DB70BD00000004024037
:10264000B08240420080404210B50F48006820F43C
:1026500040000D4908600846006840F480000860AA
:1026600001200A4908600A49C1F8B002042001F0BB
:1026700089FA002005490860042001F083FA00204F
:102680000349C1F8B00210BD00040240AC824042D0
:102690000080404210B50F48006820F440000D490A
:1026A00008600846006840F48000086000200A497D
:1026B00008600A49C1F8AC02042001F063FA012065
:1026C000054908600549C1F8AC02042001F05AFA36
:1026D00010BD000000040240B08240420080404231
:1026E00010B500241348006820F440001149086028
:1026F00008460068086001200F49086001F042FAAE
:1027000001200E49C1F8B00201F03CFA07E0601C5C
:10271000C4B2FA2C03DDFFF7BDFF012010BD06484F
:10272000803800680028F2D10349091D086000BF05
:10273000F4E7000000040240AC82404200804042C6
:1027400010B500200F4908600F48006820F4404091
:102750000D4908600846006840F480400860002089
:102760000A49C1F89C020A2001F00CFA012005492F
:1027700008600A2001F006FA00200449C1F8980216
:1027800010BD000098824042000402400080404298
:102790001CB50121022000F041FDE0200090012045
:1027A0008DF8040000208DF8060003208DF8050048
:1027B00000208DF8070069460948FFF7E0FC00207B
:1027C000084908600A2001F0DDF901200649C1F836
:1027D00094020449091D08600349C1F89C021CBD0C
:1027E00000040240948240420080404210B5002024
:1027F0000F4908600F48006820F440400D49086008
:102800000846006840F48040086001200A49C1F889
:102810009C020A2001F0B6F90120054908600A204F
:1028200001F0B0F900200449C1F8980210BD000081
:1028300098824042000402400080404270B5054644
:1028400000241648006820F44040144908600846F7
:1028500000680860002616E00020114908600A2080
:1028600001F090F901200F49C1F898026006040EAA
:102870000B487C38006808B1601CC4B20A2001F023
:1028800081F9701CC6B2082EE6DB15B9FFF7AEFF62
:1028900001E0FFF755FF204670BD00000004024034
:1028A000988240420080404270B504461548006856
:1028B00020F44040134908600846006840F4804016
:1028C0000860002010490860002517E0E0090E4963
:1028D000091D08606006040E0A2001F053F901206A
:1028E0000A49C1F898020A2001F04CF90020064973
:1028F00008600A2001F046F9681CC5B2082DE5DB26
:1029000070BD0000000402409882404200804042B6
:1029100010B50F48006820F440400D490860084693
:10292000006840F48040086001200A4908600A49B4
:10293000C1F898020A2001F025F900200549086035
:102940000A2001F01FF900200349C1F8980210BDC8
:10295000000402409C8240420080404210B50220A8
:1029600001F010F91048006820F440400E4908605A
:102970000846006840F48040086000200B49086069
:102980000B49C1F89C020A2001F0FCF8012007491C
:102990000860052001F0F6F801200549C1F89C0205
:1029A0000A2001F0EFF810BD000402409882404276
:1029B0000080404210B500241148006820F44040D7
:1029C0000F4908600846006808600A2001F0DAF83C
:1029D00001200C4908600A2001F0D4F807E0601CCF
:1029E000C4B2FA2C03DDFFF7B9FF012010BD054882
:1029F0007C3800680028F2D10249086000BFF5E782
:102A000000040240988240424CF6CC4001490860E4
:102A1000704700000030004010B500F013F810BD02
:102A200070B505460C4645F2555000F01FF8284693
:102A300000F010F8204600F013F800F003F8FFF75C
:102A4000E3FF70BD4AF6AA20014908607047000004
:102A500000300040014948607047000000300040ED
:102A6000014988607047000000300040014908605B
:102A7000704700000030004070B505460E46002447
:102A800010E02A5D02F0010104F12602D0B200F04C
:102A900017F82A5D52105100621CD0B200F010F8F5
:102AA000601CC4B2B442ECDB00F001F870BD10B59C
:102AB0000121252000F004F8142001F063F810BD76
:102AC00070B506460D460024102000F0F2F8C8202C
:102AD00001F058F8FFF71CFF7820FFF7E5FEFFF73D
:102AE00069FF044604B110E03046FFF7DDFEFFF752
:102AF00061FF044604B108E02846FFF7D5FEFFF762
:102B000059FF044604B100E000BFFFF727FFC820CB
:102B100001F038F870BD000010B54FF4A06000F06F
:102B20006BF80121022000F079FBA82000F0ECFFF7
:102B3000FA210420FFF774FF4FF4E13001F05CF953
:102B4000FDF7B8FCFEF732FE00F074F9FDF73AFC31
:102B5000FFF7E6F8002000F021FB01200149087092
:102B600010BD0000AA00002002480349086000BF11
:102B7000FEE700000400FA050CED00E070470000DD
:102B800070B5002100230F22C4781CB3174C2468B1
:102B900004F4E064C4F5E064C4F30721C1F1040463
:102BA000E3B20A4144789C40E1B284781440214366
:102BB0000C07210E0E4C05786155047804F01F05B2
:102BC0000124AC4005786D11AD0005F1E025C5F894
:102BD000004109E0047804F01F050124AC40054DD4
:102BE0000678761145F8264070BD00000CED00E037
:102BF00000E400E080E100E002490143024A116084
:102C0000704700000000FA050CED00E070B582246A
:102C10000325FFF77DFE2046FFF746FEFFF7CAFEBD
:102C200000B10EE02846FFF73FFEFFF7C3FE00B1FC
:102C300007E00020FFF738FEFFF7BCFE00B100E020
:102C400000BFFFF78BFE70BD70B5044682250126DC
:102C5000FFF75EFE2846FFF727FEFFF7ABFE00B149
:102C600010E03046FFF720FEFFF7A4FE00B109E0B8
:102C700004F00101881CFFF717FEFFF79BFE00B16F
:102C800000E000BFFFF76AFE70BD70B50024FFF7DB
:102C90003FFEE1252846FFF707FEFFF78BFE0020E9
:102CA000FFF7CCFD0446FFF7A1FDFFF757FE2046D6
:102CB00070BD70B50446FFF72BFEE0252846FFF7F0
:102CC000F3FDFFF777FE00B107E02046FFF7ECFDCC
:102CD000FFF770FE00B100E000BFFFF73FFE70BDE0
:102CE00070472DE9F05F04460E46207800F001079A
:102CF000207800F00208207800F00409207800F025
:102D0000080A207800F0100B002537B1012528466D
:102D1000FFF7CFFF012000F015FFB8F1000F06D03C
:102D200002252846FFF7C5FF012000F00BFFB9F18F
:102D3000000F06D004252846FFF7BBFF012000F056
:102D400001FFBAF1000F06D008252846FFF7B1FFB2
:102D5000012000F0F7FEBBF1000F06D01025284639
:102D6000FFF7A7FF012000F0EDFEFFF78EFFA8425E
:102D700002D00020BDE8F09F35B16422314600202A
:102D8000FDF789FA6420F5E70020F3E72DE9F05F0D
:102D900004460E46207800F00107207800F0020873
:102DA000207800F00409207800F0080A207800F06C
:102DB000100B002537B101252846FFF77AFF0120C7
:102DC00000F0C0FEB8F1000F06D002252846FFF73C
:102DD00070FF012000F0B6FEB9F1000F06D0042507
:102DE0002846FFF766FF012000F0ACFEBAF1000FA5
:102DF00006D008252846FFF75CFF012000F0A2FE60
:102E0000BBF1000F06D010252846FFF752FF012026
:102E100000F098FEFFF739FFA84202D00020BDE87D
:102E2000F09F2DB1642231460020FDF782FAF6E7CB
:102E30000020F4E71CB501210D2000F0EFF954202B
:102E4000009000208DF8040001208DF8060003207A
:102E50008DF8050000208DF8070069460F48FFF740
:102E60008EF94FF4A050009069460D48FFF787F99E
:102E70004FF44070009001208DF807006946084823
:102E8000FFF77DF969460748FFF779F94FF40040ED
:102E9000009069460148FFF772F91CBD000C024022
:102EA00000000240000802402DE9F0474021274879
:102EB000FFF7D0F9054610212448FFF7CBF9064665
:102EC00004212248FFF7C6F907464FF480512048F5
:102ED000FFF7C0F980464FF480611D48FFF7BAF94B
:102EE00081461C48007818B900250120194908704E
:102EF0001948007818B900260120174908701748AA
:102F0000007818B900270120144908701448007887
:102F100020B94FF0000801201149087011480078CD
:102F200020B94FF0000901200E49087045F0E0007B
:102F300040EA460040EA870040EAC80040EA09103B
:102F4000C043C4B22046BDE8F0870000000C024038
:102F500000000240A5000020A6000020A7000020DD
:102F6000A8000020A90000202DE9F0474FF40071CF
:102F70007748FFF76FF904464FF480717448FFF704
:102F800069F905464FF400717248FFF763F9064688
:102F90004FF480716F48FFF75DF907464FF4004129
:102FA0006D48FFF757F9804644F0E00040EA4500DD
:102FB00040EA860040EAC70040EA0810C04300F03B
:102FC000FF094FF400716248FFF744F9634909783B
:102FD000884216D04FF400715D48FFF73BF980B985
:102FE0001E2000F0AFFD4FF400715948FFF732F991
:102FF00038B90120FFF75DFE012000F0A3FDFFF7C7
:1030000005FE4FF480715248FFF724F954490978BE
:10301000884216D04FF480714D48FFF71BF980B9F4
:103020001E2000F08FFD4FF480714948FFF712F920
:1030300038B90220FFF73DFE012000F083FDFFF7C5
:10304000E5FD4FF400714348FFF704F9454909785D
:10305000884216D04FF400713E48FFF7FBF880B964
:103060001E2000F06FFD4FF400713A48FFF7F2F8B0
:1030700038B90420FFF71DFE012000F063FDFFF7C3
:10308000C5FD4FF480713348FFF7E4F836490978FD
:10309000884216D04FF480712E48FFF7DBF880B9D4
:1030A0001E2000F04FFD4FF480712A48FFF7D2F840
:1030B00038B90820FFF7FDFD012000F043FDFFF7C0
:1030C000A5FD4FF400412448FFF7C4F827490978CB
:1030D000884216D04FF400411F48FFF7BBF880B973
:1030E0001E2000F02FFD4FF400411B48FFF7B2F8FF
:1030F00038B91020FFF7DDFD012000F023FDFFF7B8
:1031000085FD4FF400711248FFF7A4F813490870C9
:103110004FF480710E48FFF79DF8114908704FF485
:1031200000710C48FFF796F80E4908704FF4807153
:103130000848FFF78FF80C4908704FF40041064823
:10314000FFF788F8094908704846BDE8F087000095
:103150000000024000080240000C0240A0000020D5
:10316000A1000020A2000020A3000020A400002055
:1031700070B504460D46052C00DC04B970BD601E18
:10318000C4B20121A140C8B2FFF793FD012000F0B5
:10319000D9FC2846FFF758FD00BFEFE72DE9F047BF
:1031A000044604F00105C4F34006C4F38007C4F3E9
:1031B000C008C4F3001929460120FFF7D9FF0120F8
:1031C00000F0C0FC31460220FFF7D2FF012000F0E2
:1031D000B9FC39460320FFF7CBFF012000F0B2FC19
:1031E00041460420FFF7C4FF012000F0ABFC494634
:1031F0000520FFF7BDFF012000F0A4FCBDE8F0872B
:10320000002101604160704710B503460C46DC6048
:103210009A601846FFF7F4FF10BD000029B1064A76
:1032200012680243044B1A6004E0034A12688243A6
:10323000014B1A60704700003038024029B1064A3D
:1032400012680243044B1A6004E0034A1268824386
:10325000014B1A607047000044380240F0B500216D
:1032600000220024022500260223324F3F6807F087
:103270000C0121B1042905D0082937D105E02E4FD2
:10328000076036E02D4F076033E02A4F3F1F3F684D
:10329000C7F38056274F3F1F3F6807F03F036EB1CB
:1032A000264FB7FBF3F7DFF88CC0ACF1040CDCF869
:1032B00000C0CCF3881C07FB0CF40CE01E4FB7FBDE
:1032C000F3F7DFF870C0ACF1040CDCF800C0CCF30D
:1032D000881C07FB0CF4174F3F1F3F68C7F30147DB
:1032E0007F1C7D00B4FBF5F7076002E0124F07601A
:1032F00000BF00BF0F4F3F6807F0F0010909104FF2
:103300007A5C0768D74047600A4F3F6807F4E0518E
:10331000890A0B4F7A5C4768D7408760054F3F6842
:1033200007F46041490B064F7A5C4768D740C76095
:10333000F0BD0000083802400024F40000127A00BA
:103340001001002001461C48814201D20020704734
:103350001A48814201D20820F9E71948814201D276
:103360001020F4E71748814201D21820EFE71648F1
:10337000814201D22020EAE71448814201D228206C
:10338000E5E71348814201D23020E0E7114881424D
:1033900001D23820DBE71048814201D24020D6E735
:1033A0000E48814201D24820D1E70D48814201D226
:1033B0005020CCE75820CAE70040000800800008F1
:1033C00000C0000800000108000002080000040816
:1033D000000006080000080800000A0800000C08A9
:1033E00000000E0830B503460C461546002206E0E4
:1033F000184600F007F844F822001B1D521CAA4290
:10340000F6D330BD01460868704700002DE9F0474B
:1034100004460E4617464FF009080025A946B4F1A8
:10342000006F02D304F0030008B1BDE8F087FEF797
:1034300083FE0020FEF7CEFD254604EB87091948E0
:10344000854218D214E02846FFF7DCFF401C70B11B
:10345000F120FEF7B9FD2846FFF774FF82460221EE
:10346000FEF7CAFD8046B8F1090F01D002E02D1D1C
:103470004D45E8D300BFB8F1090F0CD108E0204654
:103480003168FEF731FE092800D003E0241D361D07
:103490004C45F4D300BF0120FEF79CFDFEF71AFE59
:1034A00000BFC2E70000FF1F7047000030B50022D8
:1034B0008B071C0F0F2303FA04F20B4B8C1053F8ED
:1034C00024309343084C8D1044F8253023468C104B
:1034D00053F824308C07240F00FA04F42343024CE1
:1034E0008D1044F8253030BD083801400CB500205F
:1034F000019000903448006840F480303249086000
:1035000000BF3148006800F4003000900198401C72
:103510000190009818B90198B0F5A04FF1D12A4850
:10352000006800F4003010B10120009001E000209C
:1035300000900098012846D123484030006840F0B0
:1035400080502149403108602048006840F44040E4
:103550001E4908601C48083000681B490831086093
:103560000846006840F4004008600846006840F4DF
:10357000A05008601648091F0860081F006840F046
:103580008070091F086000BF0F48006800F00070DD
:103590000028F9D040F205700E4908600A4808304A
:1035A000006820F0030008490831086008460068F8
:1035B00040F00200086000BF03480830006800F0D7
:1035C0000C000828F8D10CBD003802400070004003
:1035D00008544007003C0240042808D14FF0E02185
:1035E000096941F004014FF0E022116107E04FF05A
:1035F000E021096921F004014FF0E02211617047D8
:103600007047000010B51548006840F47000134979
:1036100008601348006840F001001149086000206C
:103620000F49083108600E4800680E4908400C49EF
:1036300008600D48091D0860081F006820F48020FC
:10364000091F0860002006490C310860FFF74EFF93
:103650004FF0006001498039086010BD88ED00E03E
:1036600000380240FFFFF6FE1030002410B50121A3
:10367000054800F010F8012801D104490870012123
:10368000014800F005F810BD00040040AB00002028
:10369000CA430282704730B502460020002300244E
:1036A000158A05EA0103958905EA010413B10CB1F5
:1036B000012000E0002030BD2DE9FE430646022730
:1036C000B846404600F042FB0446FFF74DFC00B20E
:1036D0002F490880FFF7E8FB00B22E490880012E31
:1036E00014D12D48B0F900002949B1F900108842E1
:1036F0000CD12A48B0F900002649B1F900108842DF
:1037000004D1204600F08AFABDE8FE832048B0F9D3
:103710000000214908801F48B0F900001F490880B7
:103720001B48007820701B48007860706B463A4652
:1037300021463120FDF7D0FD0546012D01DB0A2D84
:1037400004DD1348B0F900001349088010480088D0
:1037500028B90F48B0F900000F49088004E00C4870
:10376000B0F900000C4908802946684600F0EAF8E4
:103770000748B0F90000084908800648B0F9000081
:1037800006490880204600F049FA00BFBCE7000067
:103790001C0200201E020020200200202202002025
:1037A0005E49098801F0200121B15C49091D0988A1
:1037B000C8B200E070475A4909780A297BD2DFE88D
:1037C00001F00517232F353B4E52616D55280ED160
:1037D0000121544A1170544A11800021534A11802A
:1037E00001214F4A117052490988524A118063E001
:1037F000AA2803D102214A4A117004E00021494A53
:103800001170474A117057E0BB2803D10321444A85
:10381000117004E00021434A1170414A11704BE0DD
:1038200004213F4A11704149088045E005213C4A86
:1038300011703E4908803FE00621394A11703B492A
:10384000098841EA0021394A11800021364A118055
:103850003649098811B90821314A11702CE0072135
:103860002F4A117000BF30490988491C2E4A118027
:10387000114609882D4A1288914202DB0821284A04
:10388000117019E00D2805D00021264A1170244A34
:10389000117002E00921224A11700DE00A2806D0B9
:1038A0000021204A11701E4A117003E003E00A2132
:1038B0001B4A117000E000BF00BF1A49097881B1AE
:1038C0001B490A680968491C194B19601A49885430
:1038D0001946096844F20802914202D300211A46AF
:1038E00011600F4909780A2915D112490988134A2C
:1038F000134B1B7822F8131011490978491C142224
:1039000091FBF2F302FB13110D4A11700021054ADD
:103910001170034A117000BF4CE700000014014011
:1039200002010020080100200E0100200C010020EF
:10393000040100200A010020748601207CC60120B9
:103940000101002070B505460E464021094800F0EF
:1039500013F800240BE0295D064800F0BFF800BF13
:103960004021044800F01DF80128F9D1641CB4423C
:10397000F1DB70BD0014014001F40072B2F5007F6C
:1039800000D100BFCA430280704721B1828942F44E
:103990000052828104E082894DF6FF731A408281D1
:1039A000704702460020B1F5007F00D100BF1388A8
:1039B0000B400BB1012000E000207047F0B503463A
:1039C000002400260025002040F66A17B94200D1E5
:1039D00000BF1846C1F3421401F01F06012707FA81
:1039E00006F5012C01D10C3004E0022C01D110307D
:1039F00000E014301AB107682F43076002E007683F
:103A0000AF430760F0BD00002DE9FF4705460E46B5
:103A10000024A14600BFA046B08900B100BF2C8A97
:103A200024F44054F08804432C82AC8941F20C60A9
:103A30008443B08831890843718908430443AC81C9
:103A4000AC8A24F44074B0890443AC826846FFF722
:103A500005FC2048854202D01F48854202D1DDF88E
:103A60000C9001E0DDF80890A88900F4004040B116
:103A700009EBC90000EB091031684900B0FBF1F710
:103A800007E009EBC90000EB091031688900B0FBC1
:103A9000F1F76420B7FBF0F004012009642101FB79
:103AA0001078A88900F4004040B1322000EBC80033
:103AB000B0FBF1F000F00700044308E0322000EB17
:103AC00008106421B0FBF1F000F00F0004432C81DA
:103AD000BDE8FF870010014000140140C1F3080257
:103AE0008280704700BFFEE702E008C8121F08C1CD
:103AF000002AFAD170477047002001E001C1121F6F
:103B0000002AFBD17047000010B504466FF0040096
:103B1000FFF762FDE11704EB5171C1F3C701074ADA
:103B200011701046007800EB4001C1EBC0104FF659
:103B3000FF7101EAC0000249088010BD9C0000200E
:103B40009E00002070B504464FF4077094FBF0F01F
:103B5000C6B24FF4077094FBF0F100FB114085B240
:103B600004B970BD05E04FF4077000F031F8701E25
:103B7000C6B2002EF7D115B1284600F029F800BFD3
:103B8000EFE700000146114A12784A434FF0E02364
:103B90005A6100229A611A46126942F001021A61C2
:103BA00000BF4FF0E022106900F001021AB100F4EA
:103BB0008032002AF5D04FF0E022126922F0010293
:103BC0004FF0E0231A6100229A6170479C000020A8
:103BD0000146114A12884A434FF0E0235A610022FD
:103BE0009A611A46126942F001021A6100BF4FF051
:103BF000E022106900F001021AB100F48032002ABC
:103C0000F5D04FF0E022126922F001024FF0E023DC
:103C10001A6100229A6170479E00002010B50028AA
:103C200021D0114B0022001F196803E0814203D804
:103C30000A4649680029F9D152B11368841A9C4296
:103C400004D1006818441060104602E0506000E0A3
:103C5000186039B102680B1A934203D10B681A44F9
:103C600002604968416010BD2C02002010B5044676
:103C7000282221460148FFF7B5FB10BD00000108CE
:103C800010B50446282221460148FFF7BFFB10BDAE
:103C90000000010800B5A9B06846FFF7E7FF4FF044
:103CA000FF30CDF882006846FFF7EAFF0A20FFF7F1
:103CB00049FF29B000BD0000FEF72EFFFEF70AFC09
:103CC0000025FDF755FDFDF753FD01211D48FDF7CA
:103CD000A7FC02211B48FDF7A3FC1F260027002498
:103CE0000CE0601CC2B231460420FDF781FE601C6E
:103CF000C2B239460520FDF77BFE641C042CF0DBC4
:103D00001EE03220FFF73EFF642095FBF0F100FB40
:103D1000115008B9FEF780FEFCF7EAFBFDF7FCFA4C
:103D200009480078012800D10AE0B5F57A7F05DB63
:103D30000120FFF7C1FCFDF71BFD00256D1C00BF36
:103D4000DFE70000FF7F200084000020F0B50B308B
:103D5000154D20F007010024144A0FE003688B4240
:103D60000BD38B4205D95E1A43184768C3E9006735
:103D700000E04368136002C004E0021D10680028E0
:103D8000ECD12046002802D1286808B10020F0BDFF
:103D9000064A07481060074A121A22F00702C0E9D3
:103DA000002401202860D7E7300200202C020020E8
:103DB000FCCE0120F8D201200D48006840F480209C
:103DC0000B4908600A481038006840F010000849A4
:103DD00010390860032001218140064A430942F856
:103DE000231000BFBFF34F8FBFF36F8F70470000EA
:103DF00024ED00E000E200E010B588B00446314A4E
:103E000031493248FFF700FA01210420FFF706FA92
:103E100001212020FFF712FA082206212C48FEF784
:103E2000F6F9082207212A48FEF7F1F9C02006908A
:103E300002208DF81C008DF81D0000208DF81E005A
:103E400001208DF81F0006A92148FEF798F9029479
:103E50000020ADF80C00ADF80E00ADF81000ADF884
:103E600014000C20ADF8120002A91A48FFF7CCFD8F
:103E700001211848FFF789FD40211648FFF77CFD16
:103E8000012240F225511348FFF798FD47208DF895
:103E9000040002208DF8050003208DF806000120A3
:103EA0008DF8070001A8FEF76BFE002005E04FF635
:103EB000FF71094A22F81010401C1428F7DB08B0E3
:103EC00010BD0000308001004406002034060020B0
:103ED00000080240001401407CC60120FC3E00089E
:103EE0000000002034020000400200083C400008AE
:103EF00034020020C4D80100F83A00081113010868
:103F00008017323032333039303531363234313651
:103F10007A68616F796F6E6778104A6948654D738A
:103F20006F3730303058326435188118284170703E
:103F30002C5265616454656D70657261747572654B
:103F40002C6E6577416E616C6F67436F6D6D4D6F61
:103F500064652C63090530546573747A0101A115F9
:103F600006050806280B08060408060208060708C6
:103F70000F1010060806030806010807030A0705C4
:103F80000A07280A0A07040A07020A07070F120885
:103F9000200D0C08040C08020C08070C10200C1C47
:103FA000050103742C02030404195CBA09183113C7
:103FB000A1093308021ADB08294613CD0A33080485
:103FC00013C50B33080513210C3308151A590819AA
:103FD0006B111A7D0832211A8B0832221A8D082A99
:103FE0002338120D33082913110E3308301A7108C3
:103FF00032321AF508323313030F3308341A5B08D0
:1040000032401A690832411AB9083242130F102B94
:10401000084338190832481AC90832501AE90832D8
:10402000E0135D112B08E120190832E31A790832F8
:0C403000E4133912022C081AFF010110E1
:040000050800018965
:00000001FF
